:1000000000EE00F010EE07F00CEC00F0000EF86EC1
:10001000060EF76E58EF06F0EE6AE550E150FCE18F
:06002000E250FAE11200BB
:10060000004465677265652043656C6369757300B6
:100610004C4D3335205465737400000000D0010147
:100620001C0E01010101206F0101010E0101216F6A
:100630000101120E010101011E6F0101010E0101F4
:100640001F6FB5EC0AF0010101011A6F01010101F0
:100650001C6701D001D007D015C112F116C113F1EA
:1006600017C114F177D101011B0E01010101206FA7
:100670000101010E0101216F0101150E01010101AE
:100680001E6F0101010E01011F6FB5EC0AF001019F
:100690000101186F010101011B51D8B401D001D033
:1006A00032D101011D6F060E01010101196F010117
:1006B0001D51010101011B51010101011C6101D00A
:1006C00001D04FD0010101011C51010101011B5D4D
:1006D00001011D6F190E01011D5DD8A001D001D0CF
:1006E00011D0000E01010101126F000E0101010184
:1006F000136F000E01010101146F1BC11CF118C121
:100700001AF12ED00101D8900101153701011637D9
:1007100001011737010101011B07010101011B51F3
:10072000010101011C19D8B401D001D004D001018C
:100730000101192FE7D70BD00101D8900101143323
:100740000101133301011233010101011C2B0101CD
:1007500001011B51010101011C6301D001D0ECD743
:1007600054D0010101011C51010101011B19D8B430
:1007700001D001D04AD0010101011B510101010149
:100780001C5D01011D6F190E01011D5DD8A001D076
:1007900001D00DD0000E01010101156F000E010105
:1007A0000101166F000E01010101176F2ED001012A
:1007B000D8900101123701011337010114370101EB
:1007C00001011C07010101011B51010101011C195B
:1007D000D8B401D001D004D001010101192FE7D70D
:1007E0000BD00101D890010117330101163301012B
:1007F0001533010101011B2B010101011B510101F5
:1008000001011C6301D001D0ECD7010101011A5193
:10081000D8B401D001D018D0FF0E01010101121B84
:10082000FF0E01010101131BFF0E01010101141B49
:10083000010E010101011227000E01010101132324
:10084000000E010101011423010101011851D8B466
:1008500001D001D018D0FF0E01010101151BFF0EC0
:1008600001010101161BFF0E01010101171B010E01
:10087000010101011527000E010101011623000EDF
:1008800001010101172301011D6F000E010101018A
:100890001A6F01011D5101010101155101010101F1
:1008A0001227010101011651010101011323010168
:1008B000010117510101010114230101010114AFCC
:1008C00001D001D020D0FF0E01010101121BFF0E4B
:1008D00001010101131BFF0E01010101141B010E97
:1008E000010101011227000E010101011323000E75
:1008F00001010101142301011D6F010E010101011C
:100900001A6F01011D511CC123F10101120E0101D9
:100910000101216F0101010E0101226F4FEC08F06E
:10092000010101011A51D8B401D001D00CD0000E40
:1009300001010101121B000E01010101131B800EB8
:1009400001010101141B12C112F113C113F114C1F1
:1009500014F100D01200000E010101010F6F000E12
:1009600001010101106F000E01010101116F010170
:100970000D0E01010101206F0101010E0101216F26
:100980000101060E010101011E6F0101010E0101AD
:100990001F6FB5EC0AF0010101010C6F01010E0E91
:1009A00001010101206F0101010E0101216F01010F
:1009B000090E010101011E6F0101010E01011F6FEE
:1009C000B5EC0AF0010101010C1B010101010E51FE
:1009D000D8B401D001D006D0010101010D6701D0CA
:1009E00001D007D00FC106F110C107F111C108F104
:1009F0008DD0010101010E517B0F010101010D2775
:100A00000101126F070E010101010E6F0101125168
:100A10000101010106A101D001D012D001010101A3
:100A20000951010101010F27010101010A510101D1
:100A300001011023010101010B51010101011123E9
:100A40000101D89001010833010107330101063388
:100A50000101D8900101093701010A3701010B3763
:100A6000010101010E2FD4D70101126F090E0101FE
:100A700001010E6F010112510101010106A101D016
:100A800001D012D0010101010951010101010F271B
:100A9000010101010A5101010101102301010101BC
:100AA0000B510101010111230101D890010108330B
:100AB00001010733010106330101D890010111330F
:100AC0000101103301010F33010101010E2FD4D7B1
:100AD0000DC123F101010F0E01010101216F01017F
:100AE000010E0101226F4FEC08F0010101010C51D0
:100AF000D8B401D001D003D001010101118F0FC181
:100B000006F110C107F111C108F100D0120000EE8A
:100B100002F011EE0EF0050EEECFE6FFE82EFCD748
:100B2000040E010101010C6F000E01010D6F000E9A
:100B3000010101010A6F000E01010B6F31D00101AB
:100B40000E0E010101010C25E96EEA6A0101010E98
:100B5000EA220A0E01010101176F000E0101186F50
:100B600006C115F107C116F186EC09F0010101017A
:100B70001551EF6E0A0E01010101176F000E010100
:100B8000186F06C115F107C116F1EEEC08F015C19A
:100B900006F116C107F1010101010C07D8A00D07EC
:100BA0000101010107510611D8A401D001D0C7D716
:100BB000010101010829D8B40929D8A401D001D024
:100BC00015D004D0010101010A4B0B2B01010E0EBF
:100BD000010101010A25E96EEA6A0101010EEA221A
:100BE000EF50D8B401D001D0EDD70FD001010101F1
:100BF00008510508010101010A6F010101010951B4
:100C0000D8A0E82A000801010B6F0101010107AF1C
:100C100001D001D012D00101136F010E01010101B9
:100C2000166F010113510101146F2D0E0101010115
:100C3000156F0101145190EC0BF00AC10CF10BC1BE
:100C40000DF1010101010D51800A800F050ED8B48C
:100C50000C5DD8A001D001D001D029D00101136FC3
:100C6000010E01010101166F0101135101010E0E68
:100C7000010101010C25E96EEA6A0101010EEA2277
:100C8000EF50300F01010101156F90EC0BF00101E5
:100C900001010C4B0D2B010101010D51800A800F48
:100CA000050ED8B40C5DD8A001D001D0D7D7120062
:100CB000640E01010101066F000E0101076F17ECC0
:100CC0000DF00101046F010E01010101066F010128
:100CD00004514EEC0BF02AEC0DF00101046F000EF4
:100CE00001010101166F010104510101056F010E9F
:100CF00001010101156F0101055190EC0BF0100E7F
:100D000001010101066F060E0101076F47EC0CF0AF
:100D10000101046F010E01010101076F010104517E
:100D20000101056F040E01010101066F010105516A
:100D3000D7EC0CF0010E01010101066F060E010156
:100D4000076F47EC0CF00101046F000E0101010177
:100D5000066F010104516EEC0CF006C102F107C1EF
:100D600003F102C106F103C107F10CEC0CF006C15E
:100D700006F107C107F108C108F13F0E01010101A9
:100D8000096FFA0E010101010A6F3E0E0101010116
:100D90000B6FABEC04F006C106F107C107F108C107
:100DA00008F1CFEC0BF006C114F107C115F108C131
:100DB00016F1ADEC07F014C100F115C101F101010C
:100DC000046F010E01010101076F010104510101CE
:100DD000056F000E01010101066F01010551D7ECFD
:100DE0000CF0030E01010101086F000E0101096FF3
:100DF00000C106F101C107F187EC05F0E80E010121
:100E00000101066F030E0101076F17EC0DF09BD770
:100E100000EF00F001011751141115111611D8A49B
:100E200001D001D00DD0000E01010101146F000EA0
:100E300001010101156F000E01010101166F8CD037
:100E400001011D6F000E01010101186F01011D510B
:100E50000101010117AF01D001D018D0010101013A
:100E6000171F0101161F0101151F0101146D000E4E
:100E700001011523010116230101172301011D6F33
:100E8000010E01010101186F01011D5101011D6FCA
:100E90008E0E01010101196F01011D510DD00101DB
:100EA000D8900101173301011633010115330101F7
:100EB000143301010101192B000E01010101141568
:100EC00001011D6F000E01010101151501011E6FC9
:100ED000000E01010101161501011F6FFF0E010136
:100EE000010117150101206F010120511D111E1173
:100EF0001F11D8A401D001D0D2D714C11AF115C145
:100F00001BF116C11CF119C123F101011A0E0101D7
:100F10000101216F0101010E0101226F4FEC08F068
:100F2000010101011851D8B401D001D00ED01AC16D
:100F300021F11BC122F11CC123F1F8EC0CF021C1FD
:100F40001AF122C11BF123C11CF11AC114F11BC1FA
:100F500015F11CC116F100D012000101190E01019A
:100F60000101206F0101010E0101216F0101140E29
:100F7000010101011E6F0101010E01011F6FB5EC9E
:100F80000AF001010101186F010101011451010171
:100F900001011A6F01010101155101011B6F0101CE
:100FA000165101011C6F01011D6B8E0E0101010123
:100FB000195F0101010119AF01D001D026D0010153
:100FC00001011951800A8F0FD8B001D001D00ED085
:100FD000000E01010101146F000E0101156F000EDA
:100FE0000101166F000E0101176F58D00101D89052
:100FF00001011D3301011C3301011B3301011A33AF
:1010000001010101193FF2D729D01F0E0101010191
:10101000196501D001D00ED0000E01010101146F3D
:10102000000E0101156F000E0101166F000E010187
:10103000176F34D00DD00101D89001011A3701018A
:101040001B3701011C3701011D370101010119077F
:1010500001010101196701D001D0EDD701010101A2
:101060001851D8B401D001D010D0010101011D1FC9
:1010700001011C1F01011B1F01011A6D000E01015E
:101080001B2301011C2301011D231AC114F11BC1E3
:1010900015F11CC116F11DC117F100D0120001019C
:1010A00001012351D8B401D001D00BD021C1E9FFF7
:1010B00022C1EAFFEE50EE10ED10D8A401D001D00D
:1010C0000CD021C1E9FF22C1EAFF000EEE6E000E36
:1010D000EE6E000EED6EED5280D00DD001010101DB
:1010E000232B21C1E9FF22C1EAFFEC52EC52D89038
:1010F000ED32ED32EF3221C1E9FF22C1EAFFEE52BB
:10110000EE52FE0EED14D8A401D001D0E7D716D0D0
:1011100001010101232B21C1E9FF22C1EAFFEE2ACF
:10112000000EEE22ED22ED5221C1E9FF22C1EAFFBD
:10113000EC52EC52D890ED32ED32EF3221C1E9FFA2
:1011400022C1EAFFEE52EE52FF0EED14D8A401D0F8
:1011500001D0DED70CD001010101230721C1E9FF35
:1011600022C1EAFFD890EE36EE36ED36ED5221C1BF
:10117000E9FF22C1EAFFEECF24F1EECF25F1EECF59
:1011800026F1010125AF01D001D0E5D70101010110
:1011900023B101D001D00BD021C1E9FF22C1EAFF68
:1011A000FF0EEE167F0EEE16FF0EED16ED5201014C
:1011B000D89023330101010123510101266F256BD2
:1011C000246B21C1E9FF22C1EAFF01012451EE1283
:1011D0002551EE122651ED12ED52120001011D6F44
:1011E000000E010101011A6F01011D5101010101F0
:1011F00018AF01D001D00FD001010101176D01011D
:10120000181FD8B0182B01011D6F010E010101013B
:101210001A6F01011D510101010116AF01D001D06A
:101220000BD001010101156D0101161FD8B0162B5D
:10123000010E010101011A1B000E010101011B6FCA
:10124000000E01011C6F0101010118511711D8B4E2
:1012500001D001D047D001011D6F010E0101010134
:10126000196F01011D5109D00101D89001011737F3
:101270000101183701010101192B0101010118AF0A
:1012800001D001D0F1D70101D89001011B37010134
:101290001C3701010101175101010101155D010117
:1012A00001011851010101011659D8A001D001D046
:1012B0000FD001010101175101010101155F010169
:1012C0000101185101010101165B010101011B819E
:1012D0000101D89001011833010117330101010107
:1012E000192FD1D7010101011A51D8B401D001D071
:1012F00007D0010101011B6D01011C1FD8B01C2B7F
:101300001BC115F11CC116F100D0120001011B6FA9
:10131000000E01010101196F01011B5101010101C1
:1013200016AF01D001D00FD001010101156D0101EF
:10133000161FD8B0162B01011B6F010E0101010110
:10134000196F01011B510101010118AF01D001D03A
:1013500007D001010101176D0101181FD8B0182B2A
:101360000101010118511711D8B401D001D03ED0AC
:1013700001011B6F010E010101011A6F01011B51D7
:1013800009D00101D8900101173701011837010177
:1013900001011A2B0101010118AF01D001D0F1D7D1
:1013A00001010101175101010101155D0101010157
:1013B0001851010101011659D8A001D001D00CD05B
:1013C00001010101175101010101155F0101010135
:1013D000185101010101165B0101D8900101183378
:1013E00001011733010101011A2FDAD701010101AF
:1013F0001951D8B401D001D007D001010101156DF8
:101400000101161FD8B0162B15C115F116C116F122
:1014100000D0120001010F0E01010101176F01013F
:10142000010E0101186F0CC114F10DC115F10EC1AF
:1014300016F160EC0AF00101010110AF01D001D0FA
:101440000DD0000E010101010C6F000E0101010120
:101450000D6F000E010101010E6F31D0150E01015B
:1014600001010F5D000E01011059D8A001D001D07B
:1014700007D00CC10CF10DC10DF10EC10EF11FD042
:101480000CC114F10DC115F10EC116F1ADEC07F050
:1014900014C114F115C115F116C116F117C117F1D8
:1014A0000AEC07F014C111F115C112F116C113F1C4
:1014B00011C10CF112C10DF113C10EF100D01200D7
:1014C0000101010114510101151101011611D8A4E6
:1014D00001D001D009D017C1E9FF18C1EAFF000E01
:1014E000EE6E000EED6E40D0010116517F0B010132
:1014F000196FD8900101193501011A6F01011B6B99
:1015000001011B3717C1E9FF18C1EAFF1AC1EEFF3D
:101510001BC1EDFF01011535E836010B0101196F03
:101520000101195117C1E9FF18C1EAFFEE12000EBF
:10153000ED1217C1E9FF18C1EAFF820EEE26FF0E79
:10154000ED220101168101011683010116850101B9
:101550001687010116890101168B0101169D0B00EA
:101560000E000101159F00D012001EC1E9FF1FC12E
:10157000EAFF010EEB34020EEB3401010101226F90
:1015800020C1E9FF21C1EAFF010122C1EFFF0101F2
:101590000101226701D001D00DD01EC1E9FF1FC19A
:1015A000EAFF000EEE6E000EEE6E000EED6EED52D6
:1015B000000E2FD00101236F000E01010101226FE7
:1015C000010123511EC1E9FF1FC1EAFF010EEB8E8D
:1015D0001EC1E9FF1FC1EAFFEECF23F1EECF24F1D8
:1015E000EECF25F1010125AF01D001D003D00101DB
:1015F0000101222B1EC1E9FF1FC1EAFFFF0EEE16FB
:10160000FF0EEE16000EED16ED5201010101225102
:1016100000D0120001011D6F000E010101011C6FBD
:1016200001011D510F0E95128A848A9200D08C8878
:1016300000D083CF1CF1010101011C39F00B010125
:1016400001011C6F00D08C9800F000D000D08C8875
:1016500000D083CF1BF10F0E010101011B17010107
:1016600001011C51010101011B11010101011C6F4C
:10167000010101011C51800B010101011A6F00D011
:101680008C9800F000D000D0010101011A6701D050
:1016900001D0CDD78A94F00E95161200C30E010129
:1016A000076F8E0EE82EFED7072FFCD7F00E95168B
:1016B000959893929394F00E8C168C988A948A92B3
:1016C00000F08C888C8200F000D000D08C9800F064
:1016D00000D000D00AEC0BF00101076F000E0101F1
:1016E0000101166F010107510101010106510C09A9
:1016F00001010101156F90EC0BF00101076F000E65
:1017000001010101166F010107510101086F280E47
:1017100001010101156F0101085190EC0BF012005D
:101720000101010115390F0B01010101176F0101C1
:10173000010115510F0B01010101186F0101010198
:10174000166701D001D002D08A9201D08A8200D0DF
:101750008C888C50F00B010101011711010101016E
:10176000196F19C18CFF00F000D000D08C9800F0E8
:1017700000D000D08C888C50F00B010101011811B1
:1017800001010101196F19C18CFF00F000D000D0D8
:101790008C9800F000D000D00AEC0BF0120006C1CB
:1017A0000CF107C10DF108C10EF10AEC0AF00CC1F1
:1017B0000FF10DC110F10EC111F106C10CF107C1FD
:1017C0000DF108C10EF1B5EC0CF00CC109F10DC121
:1017D0000AF10EC10BF109C10EF10AC10FF10BC1E3
:1017E00010F10101060E010101010C6F0101010E52
:1017F00001010D6F93EC0CF006C10CF107C10DF166
:1018000008C10EF10AEC0AF00CC106F10DC107F196
:101810000EC108F100D012000101010107510611AB
:10182000D8A401D001D00DD0000E01010101066F36
:10183000000E01010101076F000E01010101086F97
:1018400025D00101010106C109F10101010107C112
:101850000AF1010101010B6B01010C6F8E0E0101F8
:101860000101236F01010C510101090E0101010168
:10187000216F0101010E0101226F4FEC08F009C137
:1018800006F10AC107F10BC108F100D0120018D00F
:101890000101086F010E01010101166F01010851DC
:1018A000010106C1F6FF010107C1F7FF08000101B0
:1018B000F5CF15F190EC0BF001010101064B072B60
:1018C000010106C1F6FF010107C1F7FF0800F5504D
:1018D0000009D8A401D001D0DBD712000D0E010100
:1018E0000101066501D001D008D0000E01010101FF
:1018F000066F000E0101076F15D0000EC26E0101C8
:1019000001010645E846FC0BC26EC280C28200D0CF
:10191000C2B201D001D0FCD7C290C3CF06F1C4CF70
:1019200007F100D012000EC115F10FC116F110C160
:1019300017F10CC1E9FF0DC1EAFF0101EECF12F171
:101940000101EECF13F10101EDCF14F10EEC03F024
:101950000CC1E9FF0DC1EAFF12C1EEFF13C1EEFF9A
:1019600014C1EDFFED5200D01200000E0101010183
:101970000F1B000E01010101101B800E010101016E
:10198000111B0FC115F110C116F111C117F10CC1D6
:1019900012F10DC113F10EC114F10EEC03F012C1DE
:1019A0000CF113C10DF114C10EF100D01200280E7C
:1019B00001010101066101D001D019D0010101012D
:1019C0000751D8B401D001D003D001010101068D27
:1019D00001010101068F0101086F000E01010101E3
:1019E000166F0101085106C115F190EC0BF01200C1
:1019F0000101010121510101221101012311D8B47A
:101A000001D001D00CD0000E01010101211B000EFC
:101A100001010101221B800E01010101231B21C1D3
:101A200021F122C122F123C123F100D0120009D0FB
:101A3000A60EE82EFED700D0010101010607D8A0AE
:101A400007070101010107510611D8A401D001D0F7
:101A5000EFD712000101066F8A0EC06E0101065118
:021A6000120072
:020000040030CA
:0A00000000021F1E0081C1000FC0A6
:00000001FF
